:040000008A15002835
:10000800FF00030E83018316EB000A08EC008A0147
:1000180070088312A1007108A0000408A2008316CA
:100028008C1E9C2883128C1E9C281A088316EF00AD
:100038008312981C2D28181218163B08013EF00050
:1000480000300318013E3C07F1007008BB0071083E
:10005800BC00181D4128981398171A088316EF003A
:1000680083123B08013EF00000300318013E3C07B4
:10007800F1007008BB007108BC0083166F080D3AC8
:100088000319572880302406F0008030003A7002A7
:10009800031D50283F302302031857286F08133ACE
:1000A800031957287B2883120616181283168C12F8
:1000B8008312BD1683166F080D3A031968286F0856
:1000C800133A031968286D282308A53E8400800187
:1000D8007A286F083B3A03197A282308A53E84003A
:1000E8006F0880002308ED002408EE009C286F08A4
:1000F8003B3A03199C282308A53E84006F0880001A
:100108006D08013EF00000300318013E6E07F10053
:100118007008ED007108EE002308013EF000003081
:100128000318013E2407F1007008A3007108A40019
:1001380083160C1CC02883120C1CC0280C100B3012
:100148008F00DC308E00013083162102F000003071
:10015800031C013E2202F1007008A1007108A200F0
:1001680000302202031DBA28013021020318C028DA
:1001780083123D1683160C1083122108F000200804
:10018800F1002208840083166C088A006B0E830035
:06019800FF0E7F0E0900BE
:10019E00831603131419DD281F301105F1007108A1
:1001AE00003A031DDD280130F000DE28F0010800C2
:0E01BE00831603136A088A006908820008008D
:1001CC00831203132D080317960003132E0803172D
:1001DC00970003132F080317980003133008031715
:1001EC00990003138C1183169115831203138C1928
:1001FC0028292D082E042F0430040319272903174E
:10020C001608170418041904031D1D2903136B0881
:10021C00840003308000840A69088316E900831285
:10022C006A088316EA00DF208A110A122829013095
:10023C00831203179602031C9702031C9802031CDB
:10024C009902FB2883120313130803179500031359
:10025C002408003A031D3529831691163729831675
:10026C00911283128C118316111683122D08031709
:10027C00960003132E080317970003132F08031778
:10028C009800031330080317990003138C1977296E
:10029C002D082E042F043004031976290317160891
:1002AC00170418041904031D6C2903136B0884002C
:1002BC0003308000840A69088316E90083126A08F7
:1002CC008316EA00DF208A110A1277290130831283
:1002DC0003179602031C9702031C9802031C990235
:0C02EC004B29831203171508F0000800CE
:1002F800831203132D080317950003132E08031701
:10030800960003132F0803179700031330080317E9
:10031800980083160313911483160313911CBE29A6
:1003280083122D082E042F0430040319BD29031746
:100338001508160417041804031DB32903136B08C2
:10034800840006308000840A69088316E900831255
:100358006A088316EA00DF208A110A12BE290130D2
:10036800831203179502031C9602031C9702031CB1
:0603780098029029080024
:08037E0083160313111508009A
:10038600831203138C11230893002D08031795007D
:1003960003132E080317960003132F08031797005D
:1003A600031330080317980083160313141D082A35
:1003B60083122D082E042F0430040319072A03176D
:1003C6001508160417041804031DFE2903136B08E9
:1003D600840004308000840A69088316E9008312C9
:1003E6006A088316EA00DF208A110A120130831296
:1003F6000313F000512A013003179502031C9602DD
:10040600031C9702031C9802D729831203132D0895
:100416000317950003132E080317960003132F08DE
:1004260003179700031330080317980003138C195A
:10043600482A2D082E042F0430040319472A0317CF
:100446001508160417041804031D3E2A03136B0827
:10045600840004308000840A69088316E900831248
:100466006A088316EA00DF208A110A120130831215
:100476000313F000512A013003179502031C96025C
:10048600031C9702031C9802192A83160313111BD7
:0E0496004E2AF001512A11150230F000080024
:1004A400831603139818582A0000522A831203173C
:0804B40015080313990008006C
:1004BC00831203132D080317970003132E08031739
:1004CC00980003132F080317990003133008031720
:1004DC009A00950196011608123C031D772A1508FF
:1004EC008E3C031C842ACF20700803197E2A842A90
:1004FC0083120317950A0319960A712A831203179C
:10050C0012301602031D8C2A8F301502031C912AFF
:10051C007B30F000C62A83160313111483160313C1
:10052C00111CC52A83122D082E042F043004031924
:10053C00C42A03171708180419041A04031DBB2A2C
:10054C0003136B08840005308000840A6908831645
:10055C00E90083126A088316EA00DF208A110A1266
:10056C00013083120313F000C62A013003179702DF
:10057C00031C9802031C9902031C9A02942AF00192
:02058C00080065
:0E058E00831603136A088A00690882000800B9
:10059C0083120313F801F9011030FC00710DF80DF2
:1005AC00F90D7408F8027508031C750FF90203188D
:1005BC00E62A7408F80775080318750FF907031075
:0A05CC00F00DF10DFC0BD42A08001D
:1005D600831203171008F000F00CF013F00CF01360
:1005E600F00CF013F00CF0130030F1000530F007BA
:1005F60006300318013EF107700883160313E9005D
:100606007108EA00C7228A110A12F0008312031742
:100616001108840070088000110AF2000F301005DE
:10062600F0000030F1000530F00706300318013EF7
:10063600F107700883160313E9007108EA00C72260
:100646008A110A12F00072088400700880000230D5
:0C065600831203171107840080010800C4
:100662008312031306168316A301A4018030240605
:10067200F0008030003A7002031D412B4330230208
:100682000318542B2308A53E840080012308013E51
:10069200F00000300318013E2407F1007008A300A7
:1006A2007108A400372BED01EE0183121A0883169C
:1006B200EF00A301A401EF0183121816BD120B175C
:0806C20083168C168B1708004B
:1006CA000A3083120317950052220D300317950042
:0406DA0052220800A0
:1006DE00CF3083120313DD000030DE000030DF0068
:1006EE0000305E30DA000230DB000030DC0000301B
:1006FE007C30D7000130D8000030D9000030E63011
:10070E00E6000030E7002430E8000030C330E3009C
:10071E000130E4002330E5000030BF30E00001304E
:10072E00E1000030E2000030831614139413071614
:0A073E00871538308312940008007C
:10074800C7228A110A128000840AE90A0319EA0AF0
:08075800F003031DA42B0800AF
:1007600083120317100883160313A10083120317C3
:10077000110883160313A2008B01313083129000FD
:100780000C100B308F00DC308E0083160C1483129B
:0A07900010143D12C0308B00080069
:10079A001A3083120313FB005E30FC006E30FD003A
:1007AA00FD0BD52BFC0BD52BFB0BD52B0000080022
:1007BA005E22A03083120313A300C32183120317FE
:1007CA001108F000F10170080313A300C321FF30E0
:1007DA008312031710050313A300C3217C21A13040
:1007EA0083120313A300C32183120313A401E62077
:1007FA0070089200BF21831203171208F000080044
:10080A00831203179301053013020318132C1308DC
:10081A001207840020308000930A082C130812075C
:10082A008400800193031308120794000A30F4002D
:10083A00F5011008F0001108F100CE227808F00046
:10084A007908F1003030F0070317140884007008A3
:10085A0080000A30F400F5011008F0001108F100D8
:10086A00CE227008031790007108910000307106BB
:10087A00031D412C00307006031D442C462C9303A3
:04088A00182C08001E
:10088E0083160313981690308312980083168717D9
:10089E00071383128C1E562C1A08F000502C0800D9
:1008AE0083120317920110088400000891001108AA
:1008BE00003A03196D2C1108950052220317920A63
:0E08CE00120810078400000891005E2C08003C
:1008DC0083120317100883160313E90083120317FE
:1008EC00110883160313EA00C7228A110A12F000BA
:1008FC0070080319992C831203171008831603131D
:10090C00E90083120317110883160313EA00C722A8
:10091C008A110A1283120317950052220317900AA8
:08092C000319910A6E2C08006A
:100C6C00253084000E3083120313F00015308316E8
:0A0C7C00E9000630EA00A423080096
:101000008A1136268A150730831603139F00FF3096
:101010008500FF308700071083120710F030831619
:101020008600831286018316061283120616831623
:1010300088018312880183168811831288118030F9
:10104000831681008312B901BA0100303A02031DF0
:101050002B2815303902031835283908403E840002
:101060008001B90A0319BA0A25288316A50183123B
:10107000AB01AC0140308316990018158A11472442
:101080008A1518168A1165238A150710B901BA0145
:1010900000303A02031D4E28023039020318662838
:1010A0003908F000F00D70107008253E840000082B
:1010B00003179000840A000891008A116E248A1593
:1010C00083120313B90A0319BA0A4828E430031734
:1010D0009000053091008A116E248A158312031343
:1010E0008815B901BA0100303A02031D792804308D
:1010F00039020318872806128A11CD238A1506168D
:101100008A11CD238A15B90A0319BA0A7328BE3089
:1011100003179000053091008A116E248A150C3057
:101120008316031393008A116F238A1508131A304C
:10113000FB005E30FC006E30FD00FD0B9D28FC0BBB
:101140009D28FB0B9D2800003D129A30031790004C
:10115000043091008A116E248A15383083120317E7
:101160009000053091008A116E248A1583120313B2
:101170000616AB01AC01B301B401B701B80164308C
:1011800003179000003091008A11B0238A153D1A90
:10119000CA28C728881506168A1131238A15831292
:1011A00006120A3003179000003091008A11B02314
:1011B0008A153D1AE12800000000BD1EE028E12844
:1011C000D9283D1EF3280616773003179000053006
:1011D00091008A116E248A15831203133D128A111D
:1011E000CD238A153E2ABD1E342A06162D3003173C
:1011F0009000063091008A116E248A15831603131D
:101200006D08013E83120317900000300318013E61
:10121000831603136E078312031791004030920068
:101220008A1105248A15403090008A1157248A15A6
:10123000D2309000053091008A116E248A158312F5
:1012400003132B080317900003132C0803179100B6
:10125000403092008A1105248A15403090008A118E
:1012600057248A158A1165238A15A5300317900023
:101270008A1157248A158A1165238A1508120811C4
:10128000A530B600B901BA0183166E0883123A027E
:10129000031D4E2983166D08831239020318182A7C
:1012A00008150812360884000008F1007108B5001E
:1012B00041307102031C6E293508463C031C6E291F
:1012C00041303502D6000A30D607D60D5610D60D5D
:1012D0005610D60D5610D60D5610792930303502DD
:1012E000D600D60D5610D60D5610D60D5610D60D6A
:1012F0005610B60A08160811360884000008F100D6
:101300007108B50041307102031C91293508463C33
:10131000031C9129413035028316A0000A30A00732
:1013200096293030831235028316A00020088312DC
:101330005607F0007008B500B60A70080317900051
:10134000403091008A11EB228A15403090008A11BA
:1013500057248A150F3003133305F1003408F200C7
:101360000030F20500307206031DB8290030710606
:10137000031DC6293408003C031DC0293308003C66
:101380000318C6298A1165238A15CC292E30031724
:1013900095008A1152228A158A115E228A15A03080
:1013A00083120313A3008A11C3218A150630831206
:1013B0000313F0002B08F3002C08F4007008031945
:1013C000E629F30DF40D7310FF3EDF297308EE00DC
:1013D0007408EF007408F000F1017008A3008A118E
:1013E000C3218A15FF30831203136E05A30033084F
:1013F000A3078A11C3218A15831203133508A3009A
:101400008A11C3218A158A11BF218A154130FC0037
:10141000EE30FD00FD0B0A2AFC0B0A2A00008312A5
:10142000B30A0319B40A0230B9070318BA0A4429E7
:101430008A1165238A153408003C031D212A3308CC
:101440003E3C0318342A80302C06F0008030013AEC
:101450007002031D2D2AFE302B020318322AAB0A1C
:101460000319AC0AB301B40183166F08133A031DC4
:101470003A2A3E2A831208160815CB28831206162C
:10148000943003179000053091008A116E248A155C
:1014900083120313EC01ED01B101B2010812081728
:1014A000B701B8012C083802031D582A2B0837024F
:1014B0000318F02A233003179000063091008A1198
:1014C0006E248A1583120313370803179000031341
:1014D000380803179100403092008A1105248A15BC
:1014E000403090008A1157248A158A1165238A1585
:1014F000EC01ED01B901BA0100303A02031D822A64
:10150000403039020318E92A0630F2003708F000AB
:101510003808F10072080319922AF00DF10D7010CD
:10152000FF3E8B2A70086C070317900003136D08A9
:101530000318013E7107031791008A11DD238A15F4
:1015400070080313B5002130FC007630FD00FD0B60
:10155000A72AFC0BA72A000035080317900040308B
:1015600091008A11EB228A15403090008A1157248D
:101570008A150F3003133905F1003A08F2000030E4
:10158000F20500307206031DC72A00307106031DE4
:10159000D52A3A08003C031DCF2A3908003C03181D
:1015A000D52A8A1165238A15DB2A2E300317950068
:1015B0008A1152228A154030880610308806EC0ABB
:1015C0000319ED0AB10A0319B20AB90A0319BA0AD2
:1015D0007C2A8A1165238A15B70A0319B80A522A88
:1015E0008A1165238A15081208135A3003179000D0
:1015F000053091008A116E248A1583120313310875
:101600000317900003133208031791004030920033
:101610008A1105248A15403090008A1157248A15B2
:10162000F5309000053091008A116E248A158312DE
:1016300003132B080317900003132C0803179100C2
:10164000403092008A1105248A15403090008A119A
:1016500057248A158A1165238A15803088068A11D5
:08166000CD238A152D2B332B3D
:100934000D340A34203444346534703475346934E5
:10094400733420346C346534203474346534723434
:100954006D3469346E3461346C342C342034453451
:100964006E3476346F3479346534723420346C34B4
:1009740065342034663469346334683469346534E6
:10098400723420342A342E3463347334763420346D
:100994006F34753420342A34743478347434203405
:0809A4003A340D340A3400342A
:1009AC0020344D346934633472346F3463346834B6
:1009BC006934703420344934523444344134203452
:1009CC00443465346D346F34203462346F346134A4
:1009DC007234643420343134363446343834373459
:1009EC00373420342B3420344C34433444343234B4
:1009FC00783431343634203451343D34323430345C
:0C0A0C004D3468347A340A340D34003460
:100A18002034503449344334203431343634463465
:100A280038343734373420342B3420344534453483
:100A3800503452344F344D342034323434344C34FE
:100A480043343234353436342034333432344B344E
:100A58006F3420343134383430343334303437342C
:080A680020340D340A3400347F
:100A700020342E342E342034313430342034733446
:100A800065346334203470346F34753472342034F8
:100A9000763461346C3469346434653472342034AF
:100AA0006C34273465346E3476346F3469340D34E5
:040AB0000A340034D0
:100AB4000D340A3420345434453452344D344934DA
:100AC4004E34453420340D340A34203454346F34D5
:100AD400743461346C34203442347934743465347D
:0A0AE400733420343D342034003414
:100AEE00203453346F3472347434693465342034A2
:100AFE007334753472342034543469346D3465343F
:100B0E006F34753474342034313420347334653496
:0A0B1E00633420340D340A3400342F
:100B28000D340A342034443455344D345034203490
:100B380045344534503452344F344D342034203405
:0A0B48003A3420340D340A3400342E
:100B520020344D3469346B3472346F34203443346E
:100B62002034503472346F34203437342E343234DB
:0A0B7200303420340A340D3400340E
:100B7C00203449346E34693474342034493432347A
:100B8C004334313420343434303430344B346834DE
:080B9C007A340D340A340034F0
:100BA40020346234793474346534733420342C340E
:100BB400203442346C346F3463346B342034233443
:040BC40020340034A5
:100BC8002034543465347334743420345034493404
:100BD8004E34203443345434533420340D340A34DE
:020BE8000034D7
:100BEA0020344E3462342034643465342034703412
:100BFA00613467346534733420343D34203400342E
:100C0A00303431343234333434343534363437349E
:100C1A003834393441344234433444344534463424
:0C0C2A00A9340534D63404340C340534ED
:040C36000034003452
:080C3A000034003400340034E2
:040C42000034003446
:100C460050346134673465342034233420343A34E4
:040C56002034003412
:100C5A000D340A3452346534633475342034003424
:02400E007A39FD
:020000040000FA
:10420000480065006C006C006F00200049005200FF
:1042100044004100200062006F0061007200000055
:104220005000610075006C0066006A0075006A004D
:104230006F0040006600720065006500000000002D
:104240003100360046003800370037005F00490073
:1042500072006400610062006F006100720064001F
:104260005F0046006C006F00610074005F004C004E
:10427000430044005F00520053005F00500069009B
:10428000630045004500700072006F006D005F0024
:10429000320034004C0043003200350036005F002D
:1042A0004400530031003300300037005F0031001C
:1042B000340030003600300033002E006300000070
:1042C0004D00430050003200310035003000200026
:1042D000440069007300610062006C0065006400C6
:1042E0002000420079002000520065007300650044
:1042F000740020000D000A00000000000000000013
:10430000FF00FF00FF00FF00FF00FF00FF00FF00B5
:10431000FF00FF00FF00FF00FF00FF00FF00FF00A5
:10432000FF00FF00FF00FF00FF00FF00FF00FF0095
:10433000FF00FF00FF00FF00FF00FF00FF00FF0085
:104340004D0069006B0072006F00430020003100D7
:104350003600460038003700370020004900520080
:1043600044004100200062006F00610072006400A0
:1043700020005400650073007400200050004900C4
:104380004300200045004500500052004F004D0002
:104390002000310039002D00300031002D003200A6
:1043A00030003100340020000D000A000000000041
:1043B00000000000000000000000000000000000FD
:1043C0007000610075006C0066006A0075006A008C
:1043D0006F00400066007200650065002E006600F8
:1043E00072000D000A000000FF00FF00FF00FF0048
:1043F000FF00FF00FF00FF00FF00FF00FF00FF00C5
:00000001FF
